:020000040000FA
:040800004EEF07F0C0
:1008100003B210EF05F0F2B42BEF05F09EB033EF0A
:1008200005F09EB23BEF05F0F2A81AEF04F0F2B229
:1008300025EF04F0F2A620EF04F0F2B022EF04F06E
:100840002CEF07F0F296F290FF00CD90F2929EA06E
:100850002FEF04F00101463F2FEF04F0472BA1C119
:10086000A5F1A2C1A6F1A3C1A7F1A4C1A8F19DC1A0
:10087000A1F19EC1A2F19FC1A3F1A0C1A4F199C1B0
:100880009DF19AC19EF19BC19FF19CC1A0F195C1C0
:1008900099F196C19AF197C19BF198C19CF191C1D0
:1008A00095F192C196F193C197F194C198F18DC1E0
:1008B00091F18EC192F18FC193F190C194F189C1F0
:1008C0008DF18AC18EF18BC18FF18CC190F1CECFA9
:1008D00089F1CFCF8AF146C18BF147C18CF1CF6A44
:1008E000CE6A0101466B476B9E90CD800EBC0E8E8A
:1008F0000EBA7EEF04F00E8A2CEF07F00E8C0EBEBF
:10090000BAEF04F089C18DF18AC18EF18BC18FF1EC
:100910008CC190F18DC191F18EC192F18FC193F193
:1009200090C194F191C195F192C196F193C197F163
:1009300094C198F195C199F196C19AF197C19BF133
:1009400098C19CF199C19DF19AC19EF19BC19FF103
:100950009CC1A0F19DC1A1F19EC1A2F19FC1A3F1D3
:10096000A0C1A4F1A1C1A5F1A2C1A6F1A3C1A7F1A3
:10097000A4C1A8F10101516B526B536B546B8951A7
:1009800051278A5152238B5153238C5154238D511B
:1009900051278E5152238F515323905154239151FB
:1009A00051279251522393515323945154239551DB
:1009B00051279651522397515323985154239951BB
:1009C00051279A5152239B5153239C5154239D519B
:1009D00051279E5152239F515323A0515423A1517B
:1009E0005127A2515223A3515323A4515423A5515B
:1009F0005127A6515223A7515323A8515423D890CD
:100A00005433533352335133D890543353335233D6
:100A10005133D89054335333523351332CEF07F0C2
:100A20000392030103EE00F080517F0BE92604C01E
:100A3000EFFF802B8151805D700BD8A48B8200006A
:100A40008051815D700BD8A48B9281518019D8B4EC
:100A500007902CEF07F0F2940101383F2CEF07F0DC
:100A6000392B2CEF07F09E900101463F2CEF07F049
:100A7000472B2CEF07F09E9204005CA140EF05F09D
:100A8000077C07AC5BEF05F0C274C2B455EF05F00C
:100A9000C3CFADF5C4CFAEF50501D890AE33AD33BD
:100AA000D890AE33AD335CEF05F0C3CF48F1C4CF7F
:100AB00049F15CEF05F0C28207B4C9EF05F03AC115
:100AC0003EF13BC13FF13CC140F13DC141F151C15B
:100AD00055F152C156F153C157F154C158F189C172
:100AE000A9F18AC1AAF18BC1ABF18CC1ACF18DC166
:100AF000ADF18EC1AEF18FC1AFF190C1B0F191C136
:100B0000B1F192C1B2F193C1B3F194C1B4F195C105
:100B1000B5F196C1B6F197C1B7F198C1B8F199C1D5
:100B2000B9F19AC1BAF19BC1BBF19CC1BCF19DC1A5
:100B3000BDF19EC1BEF19FC1BFF1A0C1C0F1A1C175
:100B4000C1F1A2C1C2F1A3C1C3F1A4C1C4F1A5C145
:100B5000C5F1A6C1C6F1A7C1C7F1A8C1C8F1ADC50D
:100B6000AFF5AEC5B0F5AFC5B1F5B0C5B2F5010191
:100B700048514E2749514F23E86A50230D2EC9EFA3
:100B800005F04FC14AF150C14BF14E6B4F6B506BAA
:100B9000078E0201002F2CEF07F03C0E006F0501BD
:100BA0002951000AD8B478EF06F005012951010A4D
:100BB000D8B402EF06F005012951020AD8B443EF78
:100BC00006F005012951030AD8B443EF06F00501E8
:100BD0002951040AD8B443EF06F005012951050A4A
:100BE000D8B443EF06F005012951060AD8B443EF03
:100BF00006F005012951070AD8B443EF06F0296B26
:100C000078EF06F005014D670DEF06F04E670DEF2A
:100C100006F04F670DEF06F0506711EF06F078EF22
:100C200006F051C500F152C501F153C502F154C59A
:100C300003F10101010E046F000E056F000E066F37
:100C4000000E076F04EC1CF000C151F501C152F514
:100C500002C153F503C154F5006736EF06F0016792
:100C600036EF06F0026736EF06F0036778EF06F01E
:100C70004DC551F54EC552F54FC553F550C554F508
:100C80000E8878EF06F005012A6749EF06F078EF45
:100C900006F00EBE5EEF06F00FA063EF06F0010156
:100CA0003A675AEF06F03B675AEF06F03C675AEF97
:100CB00006F03D675EEF06F063EF06F007AE63EF08
:100CC00006F075EF06F005012B2F78EF06F03C0ECD
:100CD0002B6F2A2F78EF06F00101000E556FE00E02
:100CE000566FA50E576F010E586F05012A6B0E88BF
:100CF000050105015C6B2DB77FEF06F05C810101FA
:100D00007D678AEF06F07E678AEF06F07F678AEFDD
:100D100006F080678EEF06F0BEEF06F081C100F1AD
:100D200082C101F183C102F184C103F10101010E0D
:100D3000046F000E056F000E066F000E076F04ECC7
:100D40001CF000C181F101C182F102C183F103C134
:100D500084F10067B3EF06F00167B3EF06F00267B6
:100D6000B3EF06F00367BEEF06F07DC181F17EC1EF
:100D700082F17FC183F180C184F10E80D57ED5BE22
:100D800069D0D6CF3AF1D7CF3BF138C13CF1E86A10
:100D9000E8CF3DF10F903AC100F13BC101F13CC1F8
:100DA00002F13DC103F101010A0E046F000E056F4F
:100DB000000E066F000E076F04EC1CF000AF0F80F2
:100DC000010147A7F0EF06F00E9A0E9C0E9E01015E
:100DD000000E516F600E526F3D0E536F080E546F30
:100DE00001013ABF00EF07F03B6700EF07F03C67F7
:100DF00000EF07F03D6700EF07F0F28825EF07F0FE
:100E0000F298516B526B536B546B896B8A6B8B6B83
:100E10008C6B8D6B8E6B8F6B906B916B926B936BFE
:100E2000946B956B966B976B986B996B9A6B9B6BAE
:100E30009C6B9D6B9E6B9F6BA06BA16BA26BA36B5E
:100E4000A46BA56BA66BA76BA86BD76AD66A0101CA
:100E5000386B396B2CEF07F002C0E0FF005001C087
:100E6000D8FF1000A6B232EF07F00CC0A9FF0BC0EC
:100E7000A8FFA69EA69CA684F29E550EA76EAA0E5B
:100E8000A76EA682F28EA694A6B244EF07F01200D7
:100E9000A96EA69EA69CA680A8501200076A0E6A9C
:100EA0000F6A0F010D0EC16E860EC06E030EC26E6C
:100EB0000F01280E896E130E926E080E8A6EF30EC5
:100EC000936E8B6A900E946EF18EF19E0D6A010105
:100ED0004E6B4F6B506B4A6B4B6BF29A01013A6B46
:100EE0003B6B3C6B3D6B3E6B3F6B406B416B426BB6
:100EF000436B446B456B386B396BD76AD66A0F010D
:100F0000280ED56EF28A9D90B00ECD6E0101516B08
:100F1000526B536B546B556B566B576B586B596BCD
:100F20005A6B5B6B5C6B466B476BCF6ACE6A0E9AF3
:100F30000E9C0E9E9D80760ECA6E9D8202013C0E16
:100F4000006FCC6A160E48EC07F0E8CF00F1170EE0
:100F500048EC07F0E8CF01F1180E48EC07F0E8CFB5
:100F600002F1190E48EC07F0E8CF03F1010103AFDD
:100F7000D4EF07F0FBEC1CF0160E0C6E00C10BF06A
:100F800032EC07F0170E0C6E01C10BF032EC07F0DB
:100F9000180E0C6E02C10BF032EC07F0190E0C6E3D
:100FA00003C10BF032EC07F000C17DF101C17EF10D
:100FB00002C17FF103C180F100C181F101C182F161
:100FC00002C183F103C184F11A0E48EC07F0E8CFA7
:100FD00000F11B0E48EC07F0E8CF01F11C0E48ECC5
:100FE00007F0E8CF02F11D0E48EC07F0E8CF03F15F
:100FF000010103AF2AEF08F0FBEC1CF01A0E0C6E97
:1010000000C10BF032EC07F01B0E0C6E01C10BF0AF
:1010100032EC07F01C0E0C6E02C10BF032EC07F044
:101020001D0E0C6E03C10BF032EC07F01A0E48ECEB
:1010300007F0E8CF00F11B0E48EC07F0E8CF01F114
:101040001C0E48EC07F0E8CF02F11D0E48EC07F04B
:10105000E8CF03F100C185F101C186F102C187F13A
:1010600003C188F1240EAC6E900EAB6E240EAC6EF4
:10107000080EB86E000EB06E1F0EAF6E0401806BCE
:10108000816B0F01900EAB6E0F019D8A0301806B87
:10109000816BA26B8B921FEC20F0200E48EC07F0C6
:1010A000E8CF29F505012951FF0AD8A45FEF08F020
:1010B000296B200E0C6E29C50BF032EC07F00501F0
:1010C000010E2A6F3C0E2B6F250E48EC07F0E8CF7F
:1010D00000F1260E48EC07F0E8CF01F1270E48ECAE
:1010E00007F0E8CF02F1280E48EC07F0E8CF03F153
:1010F000010103AF96EF08F0FBEC1CF0250E0C6E1F
:1011000000C10BF032EC07F0260E0C6E01C10BF0A3
:1011100032EC07F0270E0C6E02C10BF032EC07F038
:10112000280E0C6E03C10BF032EC07F000C14DF538
:1011300001C14EF502C14FF503C150F500C151F593
:1011400001C152F502C153F503C154F5290E48EC13
:1011500007F0E8CF55F505015651555DD8A055C5A6
:1011600056F505012951020A0EE181B8C3EF08F0D6
:101170000501562FC0EF08F055C556F5C3EF08F02E
:1011800081BA3EEF23F0210E48EC07F0E8CF00F1E2
:10119000220E48EC07F0E8CF01F1230E48EC07F0EF
:1011A000E8CF02F1240E48EC07F0E8CF03F101018B
:1011B00003AF09EF09F0FBEC1CF0210E0C6E00C12F
:1011C0000BF032EC07F0220E0C6E01C10BF032EC8A
:1011D00007F0230E0C6E02C10BF032EC07F0240E68
:1011E0000C6E03C10BF032EC07F0210E48EC07F057
:1011F000E8CF00F1220E48EC07F0E8CF01F1230E12
:1012000048EC07F0E8CF02F1240E48EC07F0E8CFF5
:1012100003F100C157F501C158F502C159F503C1E9
:101220005AF556EC1FF018EC1EF068EC1DF00501A5
:101230002951030A12E005012951040A1DE00501A4
:101240002951050A24E005012951060A32E0050169
:101250002951070A38E06CEF09F0A6C500F1010139
:101260000F0E001701010051000A36E00101005184
:10127000050A32E069EF09F0A6C500F101010F0E81
:10128000001701010051000A27E069EF09F005018C
:10129000A651000A21E00501A651150A1DE005012D
:1012A000A651300A19E00501A651450A15E069EF7B
:1012B00009F00501A651000A0FE00501A651300A08
:1012C0000BE069EF09F00501A651000A05E069EF9E
:1012D00009F081BA3EEF23F007900001F28EF28C04
:1012E00007B09CEF19F00EB07DEF14F00EB86FEF61
:1012F0000EF00301805181197F0BD8B49CEF19F0D7
:1013000013EE00F081517F0BE126812BE7CFE8FF40
:10131000E00BD8B49CEF19F023EE82F0A2511F0B22
:10132000D926E7CFDFFFA22BDF50780AD8A49CEFA5
:1013300019F0078081C100F182C101F183C102F17E
:1013400084C103F10101040E046F000E056F000E4D
:10135000066F000E076F04EC1CF000AFB9EF09F048
:101360000101030E816F000E826F000E836F000E6D
:10137000846F03018251720AD8B47DEF14F0825158
:10138000520AD8B47DEF14F08251750AD8B47DEFBB
:1013900014F08251630AD8B458EF16F08251690AEA
:1013A000D8B438EF11F082517A0AD8B44BEF12F06A
:1013B0008251490AD8B4D7EF10F08251500AD8B4FC
:1013C000F5EF0FF08251700AD8B438EF10F0825167
:1013D000540AD8B463EF10F08251740AD8B4A9EF5C
:1013E00010F08251730AD8B4ADEF13F08251530A52
:1013F000D8B412EF14F082514C0AD8B415EF0AF0A9
:101400008DEF16F0040114EE00F080517F0BE12601
:1014100082C4E7FF802B12000D0E826F02EC0AF0EF
:101420000A0E826F02EC0AF0120003018351300AA7
:10143000D8B4C4EF0CF003018351310AD8B44AEF99
:101440000DF003018351320AD8B49AEF0DF0030175
:101450008351330AD8B49EEF0DF003018351340A4F
:10146000D8B4ACEF0DF003018351350AD8B474EF52
:101470000EF0030183514D0AD8B43DEF0BF0030188
:1014800083516D0AD8B457EF0BF003018351490A19
:10149000D8B474EF0FF003018351500AD8B4A6EF0B
:1014A0000EF003018351540AD8B41FEF0FF003016B
:1014B0008351630AD8B477EF0BF003018351430AD9
:1014C000D8B46FEF0CF003018351730AD8B475EFF1
:1014D0000BF003018351610AD8B48AEF0AF00301CB
:1014E0008351650AD8B412EF0DF003018351450A08
:1014F000D8B420EF0DF003018351620AD8B42EEF67
:101500000DF003018351420AD8B43CEF0DF0D8A48A
:101510008DEF16F004014C0E826F02EC0AF004010C
:10152000610E826F02EC0AF018EC1EF004012C0E22
:10153000826F02EC0AF0FBEC1CF0A5C500F1010182
:101540009EEC1CF025C182F40401300E822702ECCF
:101550000AF026C182F40401300E822702EC0AF060
:1015600027C182F40401300E822702EC0AF0040144
:101570002C0E826F02EC0AF0FBEC1CF0A6C500F109
:1015800001019EEC1CF025C182F40401300E82277B
:1015900002EC0AF026C182F40401300E822702EC2C
:1015A0000AF027C182F40401300E822702EC0AF00F
:1015B00004012C0E826F02EC0AF0FBEC1CF0A7C5B4
:1015C00000F101019EEC1CF025C182F40401300EF3
:1015D000822702EC0AF026C182F40401300E822731
:1015E00002EC0AF027C182F40401300E822702ECDB
:1015F0000AF004012C0E826F02EC0AF0FBEC1CF0E6
:10160000A8C500F101019EEC1CF025C182F4040183
:10161000300E822702EC0AF026C182F40401300E5B
:10162000822702EC0AF027C182F40401300E8227DF
:1016300002EC0AF004012C0E826F02EC0AF0FBECC3
:101640001CF0ADC500F101019EEC1CF025C182F437
:101650000401300E822702EC0AF026C182F4040154
:10166000300E822702EC0AF027C182F40401300E0A
:10167000822702EC0AF0A2EF0EF03CEC1DF084C3CE
:1016800027F149EC1DF0C0EC1CF0200E0C6E00C1DF
:101690000BF032EC07F000C129F505012951000AD1
:1016A00006E005012951010A02E0BEEC1EF004012A
:1016B0004C0E826F02EC0AF004014D0E826F02ECB8
:1016C0000AF004012C0E826F02EC0AF0FBEC1CF015
:1016D00029C500F19EEC1CF027C182F40401300EF4
:1016E000822702EC0AF0A2EF0EF03EEF23F0040195
:1016F0004C0E826F02EC0AF00401630E826F02EC62
:101700000AF068EC1DF004012C0E826F02EC0AF066
:101710008CEC0BF0A2EF0EF0FBEC1CF0ABC500F173
:101720000101003B0F0E00179EEC1CF027C182F454
:101730000401300E822702EC0AF0ABC500F1010172
:101740000F0E010100179EEC1CF027C182F404016A
:10175000300E822702EC0AF004012D0E826F02EC9B
:101760000AF0AAC500F10101003B0F0E00179EEC24
:101770001CF027C182F40401300E822702EC0AF02B
:10178000AAC500F101010F0E010100179EEC1CF02B
:1017900027C182F40401300E822702EC0AF0040112
:1017A0002D0E826F02EC0AF0A9C500F10101003B89
:1017B0000F0E00179EEC1CF027C182F40401300EBE
:1017C000822702EC0AF0A9C500F101010F0E010108
:1017D00000179EEC1CF027C182F40401300E822712
:1017E00002EC0AF00401200E826F02EC0AF0A8C598
:1017F00000F10F0E010100179EEC1CF027C182F4CE
:101800000401300E822702EC0AF00401200E826FE0
:1018100002EC0AF0A7C500F101010101003B0F0E27
:1018200000179EEC1CF027C182F40401300E8227C1
:1018300002EC0AF0A7C500F101010F0E010100172B
:101840009EEC1CF027C182F40401300E822702ECCA
:101850000AF004013A0E826F02EC0AF0A6C500F10C
:101860000101003B0F0E00179EEC1CF027C182F413
:101870000401300E822702EC0AF0A6C500F1010136
:101880000F0E010100179EEC1CF027C182F4040129
:10189000300E822702EC0AF004013A0E826F02EC4D
:1018A0000AF0A5C500F10101003B0F0E00179EECE8
:1018B0001CF027C182F40401300E822702EC0AF0EA
:1018C000A5C500F101010F0E00179EEC1CF027C109
:1018D00082F40401300E822702EC0AF0120084C365
:1018E000E8FF0F0BE83AE8CFABF585C3E8FF0F0B35
:1018F0000501AB1387C3E8FF0F0BE83AE8CFAAF561
:1019000088C3E8FF0F0B0501AA138AC3E8FF0F0B7A
:10191000E83AE8CFA9F58BC3E8FF0F0B0501A9133F
:101920008DC3E8FF0F0BE8CFA8F58FC3E8FF0F0BBF
:10193000E83AE8CFA7F590C3E8FF0F0B0501A7131E
:1019400092C3E8FF0F0BE83AE8CFA6F593C3E8FF90
:101950000F0B0501A61395C3E8FF0F0BE83AE8CF7C
:10196000A5F596C3E8FF0F0B0501A513C7EC1DF005
:1019700004014C0E826F02EC0AF00401430E826FE8
:1019800002EC0AF081EF0BF0FFEC22F0FBEC1CF014
:101990002DC500F19EEC1CF004014C0E826F02EC90
:1019A0000AF00401300E826F02EC0AF004012C0EE2
:1019B000826F02EC0AF025C182F40401300E822706
:1019C00002EC0AF026C182F40401300E822702ECF8
:1019D0000AF027C182F40401300E822702EC0AF0DB
:1019E00004012C0E826F02EC0AF0FBEC1CF02EC5F9
:1019F00000F19EEC1CF025C182F40401300E822718
:101A000002EC0AF026C182F40401300E822702ECB7
:101A10000AF027C182F40401300E822702EC0AF09A
:101A2000A2EF0EF004014C0E826F02EC0AF00401EA
:101A3000650E826F02EC0AF0A7EC1FF0A2EF0EF029
:101A400004014C0E826F02EC0AF00401450E826F15
:101A500002EC0AF0C4EC1FF0A2EF0EF004014C0EF1
:101A6000826F02EC0AF00401620E826F02EC0AF04F
:101A7000FEEC1FF0A2EF0EF004014C0E826F02ECA0
:101A80000AF00401420E826F02EC0AF0E1EC1FF052
:101A9000A2EF0EF004014C0E826F02EC0AF004017A
:101AA000310E826F02EC0AF004012C0E826F02EC00
:101AB0000AF025C500F126C501F127C502F128C5A8
:101AC00003F10101100E046F000E056F000E066F8A
:101AD000000E076F32EC1CF09EEC1CF022C182F469
:101AE0000401300E822702EC0AF023C182F40401C3
:101AF000300E822702EC0AF024C182F40401300E79
:101B0000822702EC0AF025C182F40401300E8227FC
:101B100002EC0AF026C182F40401300E822702ECA6
:101B20000AF027C182F40401300E822702EC0AF089
:101B3000A2EF0EF069EC20F08DEF16F004014C0ED0
:101B4000826F02EC0AF00401330E826F02EC0AF09D
:101B50009FEC20F054EF0DF004014C0E826F02EC6C
:101B60000AF00401340E826F02EC0AF004012C0E1C
:101B7000826F02EC0AF03CEC1DF084C31EF185C3B9
:101B80001FF186C320F187C321F188C322F189C3E5
:101B900023F18AC324F18BC325F18CC326F18DC3B5
:101BA00027F101011D6B49EC1DF0C0EC1CF0100E7B
:101BB000046F000E056F000E066F000E076F13EC2A
:101BC0001CF000C121F501C122F502C123F503C1BA
:101BD00024F5B2EC22F02EC5A5F52FC5A6F530C52B
:101BE000A7F531C5A8F532C5A9F533C5AAF534C5A1
:101BF000ABF58CEC0BF004012C0E826F02EC0AF0BA
:101C000035C500F136C501F137C502F138C503F11C
:101C10000101000E046F000E056F010E066F000E2D
:101C2000076F32EC1CF09EEC1CF01D671AEF0EF0F3
:101C30001FEF0EF004012D0E826F02EC0AF024C19A
:101C400082F40401300E822702EC0AF025C182F4EE
:101C50000401300E822702EC0AF004012E0E826F7E
:101C600002EC0AF026C182F40401300E822702EC55
:101C70000AF027C182F40401300E822702EC0AF038
:101C800004012C0E826F02EC0AF0FBEC1CF039C54B
:101C900000F13AC501F1B7EC17F004012C0E826F88
:101CA00002EC0AF0FBEC1CF03BC500F19EEC1CF0D2
:101CB00025C182F40401300E822702EC0AF026C10D
:101CC00082F40401300E822702EC0AF027C182F46C
:101CD0000401300E822702EC0AF0A2EF0EF00E98FB
:101CE0009FEC20F0A2EF0EF004014C0E826F02EC8C
:101CF0000AF00401350E826F02EC0AF004012C0E8A
:101D0000826F02EC0AF0FBEC1CF00784AFC500F117
:101D100007949EEC1CF025C182F40401300E82274A
:101D200002EC0AF026C182F40401300E822702EC94
:101D30000AF027C182F40401300E822702EC0AF077
:101D4000A2EF0EF00CEC0AF08DEF16F004014C0E31
:101D5000826F02EC0AF00401500E826F02EC0AF06E
:101D600004012C0E826F02EC0AF085C31EF186C3BB
:101D70001FF187C320F188C321F189C322F18AC3EF
:101D800023F18BC324F18CC325F18DC326F18EC3BF
:101D900027F1010149EC1DF0C0EC1CF00301845156
:101DA000530A0DE0030184514D0A38E00401780E16
:101DB000826F02EC0AF00CEC0AF08DEF16F00401D1
:101DC000530E826F02EC0AF0250E0C6E00C10BF070
:101DD00032EC07F0260E0C6E01C10BF032EC07F06E
:101DE000270E0C6E02C10BF032EC07F0280E0C6EC1
:101DF00003C10BF032EC07F000C14DF501C14EF507
:101E000002C14FF503C150F500C151F501C152F5B2
:101E100002C153F503C154F583EF0FF004014D0ED9
:101E2000826F02EC0AF0290E0C6E00C10BF032EC4E
:101E300007F000C155F500C156F583EF0FF004011E
:101E40004C0E826F02EC0AF00401540E826F02EC19
:101E50000AF004012C0E826F02EC0AF084C31EF11A
:101E600085C31FF186C320F187C321F188C322F106
:101E700089C323F18AC324F18BC325F18DC326F1D5
:101E80008EC327F1010149EC1DF0C0EC1CF00101EB
:101E9000000E046F000E056F010E066F000E076F37
:101EA00013EC1CF0210E0C6E00C10BF032EC07F0AD
:101EB000220E0C6E01C10BF032EC07F0230E0C6EFB
:101EC00002C10BF032EC07F0240E0C6E03C10BF0D4
:101ED00032EC07F000C157F501C158F502C159F5C0
:101EE00003C15AF583EF0FF004014C0E826F02EC30
:101EF0000AF00401490E826F02EC0AF004012C0E74
:101F0000826F02EC0AF0250E48EC07F0E8CF00F1F2
:101F1000260E48EC07F0E8CF01F1270E48EC07F059
:101F2000E8CF02F1280E48EC07F0E8CF03F19EEC71
:101F30001CF0CAEC1AF00401730E826F02EC0AF076
:101F400004012C0E826F02EC0AF0FBEC1CF0290E4F
:101F500048EC07F0E8CF00F19EEC1CF0CAEC1AF058
:101F60000401730E826F02EC0AF004012C0E826FE2
:101F700002EC0AF051C500F152C501F153C502F15E
:101F800054C503F19EEC1CF0CAEC1AF00401730E68
:101F9000826F02EC0AF004012C0E826F02EC0AF050
:101FA000FBEC1CF056C500F19EEC1CF0CAEC1AF0DC
:101FB00004016D0E826F02EC0AF004012C0E826F98
:101FC00002EC0AF057C500F158C501F159C502F1FC
:101FD0005AC503F1A8EC16F004012C0E826F02EC36
:101FE0000AF00CEC0AF08DEF16F083C31EF184C3E7
:101FF0001FF185C320F186C321F187C322F188C375
:1020000023F189C324F18AC325F18BC326F18CC344
:1020100027F1010149EC1DF0C0EC1CF0160E0C6E0E
:1020200000C10BF032EC07F0170E0C6E01C10BF083
:1020300032EC07F0180E0C6E02C10BF032EC07F018
:10204000190E0C6E03C10BF032EC07F000C17DF1EC
:1020500001C17EF102C17FF103C180F100C181F1B4
:1020600001C182F102C183F103C184F1D7EF10F005
:1020700083C31EF184C31FF185C320F186C321F100
:1020800087C322F188C323F189C324F18AC325F1D0
:102090008BC326F18CC327F1010149EC1DF0C0EC84
:1020A0001CF000C17DF101C17EF102C17FF103C1CD
:1020B00080F100C181F101C182F102C183F103C14C
:1020C00084F1D7EF10F083C31EF184C31FF185C3E1
:1020D00020F186C321F187C322F188C323F189C38C
:1020E00024F18AC325F18CC326F18DC327F10101A8
:1020F00049EC1DF0C0EC1CF00101000E046F000E55
:10210000056F010E066F000E076F13EC1CF01A0E20
:102110000C6E00C10BF032EC07F01B0E0C6E01C10F
:102120000BF032EC07F01C0E0C6E02C10BF032EC1F
:1021300007F01D0E0C6E03C10BF032EC07F000C16E
:1021400085F101C186F102C187F103C188F1D7EFA2
:1021500010F083C31EF184C31FF185C320F186C331
:1021600021F187C322F188C323F189C324F18AC3F3
:1021700025F18CC326F18DC327F1010149EC1DF037
:10218000C0EC1CF00101000E046F000E056F010E83
:10219000066F000E076F13EC1CF000C185F101C142
:1021A00086F102C187F103C188F1D7EF10F0160E56
:1021B00048EC07F0E8CF00F1170E48EC07F0E8CF45
:1021C00001F1180E48EC07F0E8CF02F1190E48ECC7
:1021D00007F0E8CF03F19EEC1CF0CAEC1AF0040102
:1021E000730E826F02EC0AF004012C0E826F02EC77
:1021F0000AF07DC100F17EC101F17FC102F180C111
:1022000003F19EEC1CF0CAEC1AF00401730E826F0D
:1022100002EC0AF004012C0E826F02EC0AF01A0E96
:1022200048EC07F0E8CF00F11B0E48EC07F0E8CFD0
:1022300001F11C0E48EC07F0E8CF02F11D0E48EC4E
:1022400007F0E8CF03F1A8EC16F004012C0E826F22
:1022500002EC0AF085C100F186C101F187C102F1EB
:1022600088C103F1A8EC16F00CEC0AF08DEF16F023
:102270000401690E826F02EC0AF004012C0E826FD9
:1022800002EC0AF00101040E006F000E016F000E57
:10229000026F000E036F9EEC1CF020C182F404015B
:1022A000300E822702EC0AF021C182F40401300EC4
:1022B000822702EC0AF022C182F40401300E822748
:1022C00002EC0AF023C182F40401300E822702ECF2
:1022D0000AF024C182F40401300E822702EC0AF0D5
:1022E00025C182F40401300E822702EC0AF026C1D7
:1022F00082F40401300E822702EC0AF027C182F436
:102300000401300E822702EC0AF004012C0E826FC9
:1023100002EC0AF00101060E006F000E016F000EC4
:10232000026F000E036F9EEC1CF020C182F40401CA
:10233000300E822702EC0AF021C182F40401300E33
:10234000822702EC0AF022C182F40401300E8227B7
:1023500002EC0AF023C182F40401300E822702EC61
:102360000AF024C182F40401300E822702EC0AF044
:1023700025C182F40401300E822702EC0AF026C146
:1023800082F40401300E822702EC0AF027C182F4A5
:102390000401300E822702EC0AF004012C0E826F39
:1023A00002EC0AF00101180E006F000E016F000E22
:1023B000026F000E036F9EEC1CF020C182F404013A
:1023C000300E822702EC0AF021C182F40401300EA3
:1023D000822702EC0AF022C182F40401300E822727
:1023E00002EC0AF023C182F40401300E822702ECD1
:1023F0000AF024C182F40401300E822702EC0AF0B4
:1024000025C182F40401300E822702EC0AF026C1B5
:1024100082F40401300E822702EC0AF027C182F414
:102420000401300E822702EC0AF004012C0E826FA8
:1024300002EC0AF0200EF86EF76AF66A0401090051
:10244000F5CF82F402EC0AF00900F5CF82F402EC39
:102450000AF00900F5CF82F402EC0AF00900F5CF8A
:1024600082F402EC0AF00900F5CF82F402EC0AF0E3
:102470000900F5CF82F402EC0AF00900F5CF82F4EE
:1024800002EC0AF00900F5CF82F402EC0AF00CEC41
:102490000AF08DEF16F08351630AD8A48DEF16F081
:1024A0008451610AD8A48DEF16F085516C0AD8A426
:1024B0008DEF16F08651410A42E08651440A1BE036
:1024C0008651420AD8B4B2EF12F08651350AD8B418
:1024D00017EF18F08651360AD8B46CEF18F0865111
:1024E000370AD8B4D5EF18F08651380AD8B433EF8C
:1024F00019F08DEF16F00798079A04017A0E826F93
:1025000002EC0AF00401780E826F02EC0AF004017A
:10251000640E826F02EC0AF081A896EF12F00401BB
:10252000550E826F02EC0AF09BEF12F004014C0E84
:10253000826F02EC0AF00CEC0AF08DEF16F00788BF
:10254000079A04017A0E826F02EC0AF00401410E30
:10255000826F02EC0AF00401610E826F02EC0AF055
:102560008CEF12F00798078A04017A0E826F02EC52
:102570000AF00401420E826F02EC0AF00401610EBF
:10258000826F02EC0AF08CEF12F001015967D0EF74
:1025900012F05A67D0EF12F05B67D0EF12F05C6771
:1025A000E8EF12F04267DCEF12F04367DCEF12F065
:1025B0004467DCEF12F04567E8EF12F00101000E0E
:1025C000006F000E016F000E026F000E036F12000D
:1025D0000101620E046F010E056F000E066F000E02
:1025E000076F59C100F15AC101F15BC102F15CC131
:1025F00003F104EC1CF003BF6CEF13F00101000EBB
:10260000046FA80E056F550E066F020E076F59C1B5
:1026100000F15AC101F15BC102F15CC103F159C182
:1026200079F15AC17AF15BC17BF15CC17CF104ECB8
:102630001CF003BF25EF13F00101000E796FA80E07
:102640007A6F550E7B6F020E7C6F0E0E48EC07F012
:10265000E8CF0CF10F0E48EC07F0E8CF0DF1100EAB
:1026600048EC07F0E8CF0EF1110E48EC07F0E8CF88
:102670000FF14DEC1BF079C104F17AC105F17BC17A
:1026800006F17CC107F104EC1CF0078211EC1BF091
:102690004DEC1BF0079211EC1BF079C100F17AC1EF
:1026A00001F17BC102F17CC103F1079211EC1BF037
:1026B000CC0E046FE00E056F870E066F050E076FD8
:1026C00004EC1CF000C10CF101C10DF102C10EF1CE
:1026D00003C10FF1A4EF13F00101800E006F1A0E79
:1026E000016F060E026F000E036F42C104F143C179
:1026F00005F144C106F145C107F104EC1CF003AF3C
:1027000085EF13F0FBEC1CF012000E0E48EC07F006
:10271000E8CF0CF10F0E48EC07F0E8CF0DF1100EEA
:1027200048EC07F0E8CF0EF1110E48EC07F0E8CFC7
:102730000FF142C100F143C101F144C102F145C1B1
:1027400003F1078211EC1BF00CC100F10DC101F186
:102750000EC102F10FC103F112000401730E826F6A
:1027600002EC0AF004012C0E826F02EC0AF00784DE
:1027700055C159F156C15AF157C15BF158C15CF1CD
:102780003EC142F13FC143F140C144F141C145F175
:102790004AC14CF14BC14DF10794D3EC13F00CEC52
:1027A0000AF08DEF16F059C100F15AC101F15BC179
:1027B00002F15CC103F101019EEC1CF0CAEC1AF0BD
:1027C0000401630E826F02EC0AF004012C0E826F8A
:1027D00002EC0AF042C100F143C101F144C102F12F
:1027E00045C103F101019EEC1CF0CAEC1AF0040192
:1027F000660E826F02EC0AF004012C0E826F02EC6E
:102800000AF0FBEC1CF04CC100F14DC101F10101DB
:102810009EEC1CF0CAEC1AF00401740E826F02ECFC
:102820000AF012000F820401530E826F02EC0AF0CC
:1028300004012C0E826F02EC0AF083C31EF184C3E4
:102840001FF185C320F186C321F187C322F188C31C
:1028500023F189C324F18AC325F18BC326F18CC3EC
:1028600027F1010149EC1DF0C0EC1CF000C159F149
:1028700001C15AF102C15BF103C15CF18EC31EF1CB
:102880008FC31FF190C320F191C321F192C322F1B4
:1028900093C323F194C324F195C325F196C326F184
:1028A00097C327F1010149EC1DF0C0EC1CF000C1F9
:1028B00042F101C143F102C144F103C145F13CECD5
:1028C0001DF099C323F19AC324F19BC325F19CC346
:1028D00026F19DC327F1010149EC1DF0C0EC1CF06D
:1028E00000C14CF101C14DF1D3EC13F004012C0EE9
:1028F000826F02EC0AF084EF14F08251520A03E175
:102900000E8284EF14F00E928251750A03E10F8457
:102910008BEF14F00F948251550A03E10F8692EF6A
:1029200014F00F9607840FB2EFEF14F00FA4DBEF53
:1029300014F0A9C159F1AAC15AF1ABC15BF1ACC104
:102940005CF1ADC15DF1AEC15EF1AFC15FF1B0C18F
:1029500060F1B1C161F1B2C162F1B3C163F1B4C15F
:1029600064F1B5C165F1B6C166F1B7C167F1B8C12F
:1029700068F1B9C169F1BAC16AF1BBC16BF1BCC1FF
:102980006CF1BDC16DF1BEC16EF1BFC16FF1C0C1CF
:1029900070F1C1C171F1C2C172F1C3C173F1C4C19F
:1029A00074F1C5C175F1C6C176F1C7C177F1C8C16F
:1029B00078F1E3EF14F055C159F156C15AF157C1FE
:1029C0005BF158C15CF13EC142F13FC143F140C1EE
:1029D00044F141C145F14AC14CF14BC14DF107945D
:1029E0000EA011EF15F001018567FEEF14F0866768
:1029F000FEEF14F08767FEEF14F0886702EF15F022
:102A000011EF15F0C5EC12F085C104F186C105F196
:102A100087C106F188C107F104EC1CF003BF55EF34
:102A200016F0C5EC12F00101000E046F000E056FE8
:102A3000010E066F000E076F32EC1CF00FA428EF9A
:102A400015F00401750E826F02EC0AF02DEF15F0FF
:102A50000401720E826F02EC0AF004012C0E826FE8
:102A600002EC0AF09EEC1CF01D673CEF15F004012F
:102A7000200E826F3FEF15F004012D0E826F02ECE5
:102A80000AF024C182F40401300E822702EC0AF01D
:102A900025C182F40401300E822702EC0AF0040101
:102AA0002E0E826F02EC0AF026C182F40401300E71
:102AB000822702EC0AF027C182F40401300E82273B
:102AC00002EC0AF004016D0E826F02EC0AF00401C0
:102AD0002C0E826F02EC0AF042C100F143C101F1F9
:102AE00044C102F145C103F101019EEC1CF0CAECA6
:102AF0001AF00401480E826F02EC0AF004017A0E0B
:102B0000826F02EC0AF004012C0E826F02EC0AF0D4
:102B100059C100F15AC101F15BC102F15CC103F17D
:102B200001019EEC1CF0CAEC1AF00401630E826FE6
:102B300002EC0AF004012C0E826F02EC0AF059C17B
:102B400000F15AC101F15BC102F15CC103F1010165
:102B50000A0E046F000E056F000E066F000E076F61
:102B600013EC1CF0000E046F120E056F000E066FC2
:102B7000000E076F32EC1CF09EEC1CF01EC182F4BC
:102B80000401300E822702EC0AF01FC182F4040116
:102B9000300E822702EC0AF020C182F40401300ECC
:102BA000822702EC0AF021C182F40401300E822750
:102BB00002EC0AF022C182F40401300E822702ECFA
:102BC0000AF023C182F40401300E822702EC0AF0DD
:102BD00024C182F40401300E822702EC0AF00401C1
:102BE0002E0E826F02EC0AF025C182F40401300E31
:102BF000822702EC0AF026C182F40401300E8227FB
:102C000002EC0AF027C182F40401300E822702ECA4
:102C10000AF00401730E826F02EC0AF004012C0E1C
:102C2000826F02EC0AF0FBEC1CF04CC100F14DC1CC
:102C300001F1B7EC17F00EB221EF16F00EA053EF32
:102C400016F004012C0E826F02EC0AF0200EF86ED2
:102C5000F76AF66A04010900F5CF82F402EC0AF083
:102C60000900F5CF82F402EC0AF00900F5CF82F4F6
:102C700002EC0AF00900F5CF82F402EC0AF0090038
:102C8000F5CF82F402EC0AF00900F5CF82F402ECF1
:102C90000AF00900F5CF82F402EC0AF00900F5CF42
:102CA00082F402EC0AF00CEC0AF00E908DEF16F0B4
:102CB0000401630E826F02EC0AF004012C0E826F95
:102CC00002EC0AF093EC16F004012C0E826F02EC79
:102CD0000AF006EC17F004012C0E826F02EC0AF0E9
:102CE00082EC17F004012C0E826F02EC0AF0010155
:102CF000F80E006FCD0E016F660E026F030E036FAC
:102D0000A8EC16F004012C0E826F02EC0AF098EC8D
:102D100017F00CEC0AF08DEF16F00301A26B079090
:102D20000F929CEF19F0D8900E0E48EC07F0E8CF08
:102D300000F10F0E48EC07F0E8CF01F1100E48EC5F
:102D400007F0E8CF02F1110E48EC07F0E8CF03F1ED
:102D50000101000E046F000E056F010E066F000EDC
:102D6000076F32EC1CF09EEC1CF01EC182F40401D3
:102D7000300E822702EC0AF01FC182F40401300EEB
:102D8000822702EC0AF020C182F40401300E82276F
:102D900002EC0AF021C182F40401300E822702EC19
:102DA0000AF022C182F40401300E822702EC0AF0FC
:102DB00023C182F40401300E822702EC0AF024C100
:102DC00082F40401300E822702EC0AF025C182F45D
:102DD0000401300E822702EC0AF004012E0E826FED
:102DE00002EC0AF026C182F40401300E822702ECC4
:102DF0000AF027C182F40401300E822702EC0AF0A7
:102E000004016D0E826F02EC0AF01200120E48EC03
:102E100007F0E8CF00F1130E48EC07F0E8CF01F11E
:102E2000140E48EC07F0E8CF02F1150E48EC07F05D
:102E3000E8CF03F101010A0E046F000E056F000ECA
:102E4000066F000E076F13EC1CF0000E046F120EDD
:102E5000056F000E066F000E076F32EC1CF09EEC43
:102E60001CF01EC182F40401300E822702EC0AF02D
:102E70001FC182F40401300E822702EC0AF020C147
:102E800082F40401300E822702EC0AF021C182F4A0
:102E90000401300E822702EC0AF022C182F4040100
:102EA000300E822702EC0AF023C182F40401300EB6
:102EB000822702EC0AF024C182F40401300E82273A
:102EC00002EC0AF004012E0E826F02EC0AF025C11A
:102ED00082F40401300E822702EC0AF026C182F44B
:102EE0000401300E822702EC0AF027C182F40401AB
:102EF000300E822702EC0AF00401730E826F02EC9E
:102F00000AF012000A0E48EC07F0E8CF00F10B0EB1
:102F100048EC07F0E8CF01F10C0E48EC07F0E8CFE1
:102F200002F10D0E48EC07F0E8CF03F1B7EF17F010
:102F3000060E48EC07F0E8CF00F1070E48EC07F06A
:102F4000E8CF01F1080E48EC07F0E8CF02F1090ED6
:102F500048EC07F0E8CF03F1B7EF17F00101FBEC05
:102F60001CF007844AC100F14BC101F10794010133
:102F7000E80E046F800E056F000E066F000E076FDF
:102F800013EC1CF0000E046F040E056F000E066FAC
:102F9000000E076F32EC1CF0880E046F130E056FE5
:102FA000000E066F000E076F04EC1CF00A0E046F93
:102FB000000E056F000E066F000E076F32EC1CF05E
:102FC0009EEC1CF001011D67EBEF17F00401200ED1
:102FD000826FEEEF17F004012D0E826F02EC0AF003
:102FE00024C182F40401300E822702EC0AF025C1CC
:102FF00082F40401300E822702EC0AF026C182F42A
:103000000401300E822702EC0AF004012E0E826FBA
:1030100002EC0AF027C182F40401300E822702EC90
:103020000AF00401430E826F02EC0AF0120087C31B
:103030001EF188C31FF189C320F18AC321F18BC31C
:1030400022F18CC323F18DC324F18EC325F190C3EB
:1030500026F191C327F101011D6B49EC1DF0C0EC75
:103060001CF00101000E046F000E056F010E066FCB
:10307000000E076F13EC1CF00E0E0C6E00C10BF06F
:1030800032EC07F00F0E0C6E01C10BF032EC07F0C2
:10309000100E0C6E02C10BF032EC07F0110E0C6E2C
:1030A00003C10BF032EC07F004017A0E826F02ECE0
:1030B0000AF004012C0E826F02EC0AF00401350EB6
:1030C000826F02EC0AF004012C0E826F02EC0AF00F
:1030D00093EC16F09BEF12F087C31EF188C31FF12B
:1030E00089C320F18AC321F18BC322F18CC323F160
:1030F0008DC324F18EC325F190C326F191C327F12E
:1031000001011D6B49EC1DF0C0EC1CF0880E046F32
:10311000130E056F000E066F000E076F08EC1CF013
:10312000000E046F040E056F000E066F000E076F91
:1031300013EC1CF00101E80E046F800E056F000E09
:10314000066F000E076F32EC1CF00A0E0C6E00C109
:103150000BF032EC07F00B0E0C6E01C10BF032ECF1
:1031600007F00C0E0C6E02C10BF032EC07F00D0EE6
:103170000C6E03C10BF032EC07F004017A0E826F83
:1031800002EC0AF004012C0E826F02EC0AF004013A
:10319000360E826F02EC0AF004012C0E826F02ECF4
:1031A0000AF082EC17F09BEF12F087C31EF188C380
:1031B0001FF189C320F18AC321F18BC322F18CC393
:1031C00023F18DC324F18FC325F190C326F191C360
:1031D00027F1010149EC1DF0C0EC1CF0000E046F5A
:1031E000120E056F000E066F000E076F13EC1CF039
:1031F00001010A0E046F000E056F000E066F000E2F
:10320000076F32EC1CF0120E0C6E00C10BF032ECAA
:1032100007F0130E0C6E01C10BF032EC07F0140E28
:103220000C6E02C10BF032EC07F0150E0C6E03C1F0
:103230000BF032EC07F004017A0E826F02EC0AF018
:1032400004012C0E826F02EC0AF00401370E826F2B
:1032500002EC0AF004012C0E826F02EC0AF006EC7C
:1032600017F09BEF12F087C31EF188C31FF189C3CB
:1032700020F18AC321F18BC322F18CC323F18DC3CA
:1032800024F18EC325F190C326F191C327F10101EA
:103290001D6B49EC1DF0C0EC1CF0880E046F130E82
:1032A000056F000E066F000E076F08EC1CF0000E95
:1032B000046F040E056F000E066F000E076F13EC0F
:1032C0001CF00101E80E046F800E056F000E066F02
:1032D000000E076F32EC1CF0060E0C6E00C10BF0F6
:1032E00032EC07F0070E0C6E01C10BF032EC07F068
:1032F000080E0C6E02C10BF032EC07F0090E0C6EDA
:1033000003C10BF032EC07F004017A0E826F02EC7D
:103310000AF004012C0E826F02EC0AF00401380E50
:10332000826F02EC0AF004012C0E826F02EC0AF0AC
:1033300098EC17F09BEF12F081A85AEF1AF007A84B
:1033400013EF1AF00101800E006F1A0E016F060EC6
:10335000026F000E036F3EC104F13FC105F140C191
:1033600006F141C107F104EC1CF003BF5AEF1AF05B
:10337000C4EC1AF03EC100F13FC101F140C102F1BD
:1033800041C103F1078211EC1BF00CC104F10DC126
:1033900005F10EC106F10FC107F1F80E006FCD0E59
:1033A000016F660E026F030E036F04EC1CF00E0E2D
:1033B0000C6E00C10BF032EC07F00F0E0C6E01C169
:1033C0000BF032EC07F0100E0C6E02C10BF032EC79
:1033D00007F0110E0C6E03C10BF032EC07F00784FE
:1033E0000101FBEC1CF04AC100F14BC101F1079453
:1033F0000A0E0C6E00C10BF032EC07F00B0E0C6ED7
:1034000001C10BF032EC07F00C0E0C6E02C10BF098
:1034100032EC07F00D0E0C6E03C10BF032EC07F02E
:1034200007985AEF1AF007AA5AEF1AF00784010119
:10343000FBEC1CF04AC100F14BC101F10794060EF0
:103440000C6E00C10BF032EC07F0070E0C6E01C1E0
:103450000BF032EC07F0080E0C6E02C10BF032ECF0
:1034600007F0090E0C6E03C10BF032EC07F0078475
:1034700055C100F156C101F157C102F158C103F124
:103480000794120E0C6E00C10BF032EC07F0130E15
:103490000C6E01C10BF032EC07F0140E0C6E02C181
:1034A0000BF032EC07F0150E0C6E03C10BF032EC92
:1034B00007F0079A0401805181197F0B0BE09EA849
:1034C00009D014EE00F081517F0BE126E750812BEB
:1034D0000F01AD6E05012951010A13E081AA81EFA8
:1034E0001AF005012951000A0AE00EB881EF1AF01E
:1034F00005012A6781EF1AF00EB881EF1AF03EEF4E
:1035000023F081B896EF1AF018EC1EF0050129514E
:10351000020A02E096EF1AF0562F96EF1AF055C500
:1035200056F50501010E2A6F3C0E2B6F70EF09F066
:103530000CC100F10DC101F10EC102F10FC103F187
:10354000000E046F000E056F010E066F000E076F70
:1035500032EC1CF01DA1C3EF1AF01451D8B4C3EF24
:103560001AF00CC100F10DC101F10EC102F10FC141
:1035700003F1000E046F000E056F0A0E066F000EB9
:10358000076F32EC1CF0120001010C6B0D6B0E6B1F
:103590000F6B12001EC182F40401300E822702EC70
:1035A0000AF01FC182F40401300E822702EC0AF0F7
:1035B00020C182F40401300E822702EC0AF021C1FE
:1035C00082F40401300E822702EC0AF022C182F458
:1035D0000401300E822702EC0AF023C182F40401B8
:1035E000300E822702EC0AF024C182F40401300E6E
:1035F000822702EC0AF025C182F40401300E8227F2
:1036000002EC0AF026C182F40401300E822702EC9B
:103610000AF027C182F40401300E822702EC0AF07E
:1036200012000101005305E1015303E1025301E1DE
:10363000002BD4EC1BF0FBEC1CF02C51006F2D5137
:10364000016F420E046F4B0E056F000E066F000EE9
:10365000076F13EC1CF000C104F101C105F102C1B8
:1036600006F103C107F10CC100F10DC101F10EC15A
:1036700002F10FC103F107B242EF1BF008EC1CF09E
:1036800044EF1BF004EC1CF000C10CF101C10DF182
:1036900002C10EF103C10FF11200FBEC1CF04CC192
:1036A00000F14DC101F1060E48EC07F0E8CF04F13E
:1036B000070E48EC07F0E8CF05F1080E48EC07F0DC
:1036C000E8CF06F1090E48EC07F0E8CF07F104EC6B
:1036D0001CF000C118F101C119F102C11AF103C1B6
:1036E0001BF1290E046F000E056F000E066F000E11
:1036F000076F13EC1CF0EE0E046F430E056F000E07
:10370000066F000E076F08EC1CF018C104F119C118
:1037100005F11AC106F11BC107F113EC1CF000C141
:1037200010F101C111F102C112F103C113F1120E26
:1037300048EC07F0E8CF04F1130E48EC07F0E8CFAF
:1037400005F1140E48EC07F0E8CF06F1150E48EC31
:1037500007F0E8CF07F10D0E006F000E016F000EAD
:10376000026F000E036F13EC1CF0180E046F000EB6
:10377000056F000E066F000E076F32EC1CF010C1D3
:1037800004F111C105F112C106F113C107F108ECF2
:103790001CF06A0E046F2A0E056F000E066F000EF5
:1037A000076F04EC1CF01200BF0EFA6E200E2D6F96
:1037B0002C6BD8900037013702370337D8B0E5EFCC
:1037C0001BF02D2FDAEF1BF02C072D070353D8B475
:1037D00012000331070B8009326F03390F0B010F01
:1037E0002C6F80EC5FF0336F2C0580EC5FF0335D65
:1037F000335F2C6B3233D8B02C272C3332A9FAEF3D
:103800001BF033512C27120020EC1DF0D8B0120011
:1038100003510719286FE3EC1CF0D89007510319E6
:1038200028AF800F1200286B07EC1DF0D8A01DEC0C
:103830001DF0D8B01200F2EC1CF0FBEC1CF01F0ED7
:10384000296F33EC1DF00B35D8B0E3EC1CF0D8A099
:103850000335D8B01200292F21EF1CF028B10AEC53
:103860001DF01200286B0451051106110711000804
:10387000D8A007EC1DF0D8A01DEC1DF0D8B01200A8
:10388000086B096B0A6B0B6B33EC1DF01F0E296F75
:1038900033EC1DF007510B5DD8A45BEF1CF0065113
:1038A0000A5DD8A45BEF1CF00551095DD8A45BEF5D
:1038B0001CF00451085DD8A06EEF1CF00451085FA5
:1038C0000551D8A0053D095F0651D8A0063D0A5F05
:1038D0000751D8A0073D0B5FD8900081292F48EFF2
:1038E0001CF028B10AEC1DF0286B07EC1DF0D890F5
:1038F00037EC1DF007510B5DD8A48BEF1CF006517F
:103900000A5DD8A48BEF1CF00551095DD8A48BEF9C
:103910001CF00451085DD8A09AEF1CF0003F9AEF0C
:103920001CF0013F9AEF1CF0023F9AEF1CF0032BB2
:10393000D8B4120028B10AEC1DF012000101286B66
:1039400007EC1DF0D8B012003CEC1DF0200E296FE2
:10395000003701370237033711EE27F00A0E2A6FBE
:10396000E7360A0EE75CD8B0E76EE5522A2FB0EFD3
:103970001CF0292FA8EF1CF028B11D81D89012004F
:1039800001010A0E286F200E296F11EE1DF028513B
:103990002A6F0A0ED890E652D8B0E726E7322A2FCF
:1039A000CBEF1CF00333023301330033292FC5EF73
:1039B0001CF0E750FF0FD8A00335D8B012001DB19E
:1039C0000AEC1DF01200045100270551D8B0053D46
:1039D00001270651D8B0063D02270751D8B0073D50
:1039E000032712000051086F0151096F02510A6F3D
:1039F00003510B6F12000101006B016B026B036B33
:103A000012000101046B056B066B076B1200033596
:103A1000D8A012000351800B001F011F021F031FBB
:103A2000003F1AEF1DF0013F1AEF1DF0023F1AEFA1
:103A30001DF0032B282B032512000735D8A01200F8
:103A40000751800B041F051F061F071F043F30EF9F
:103A50001DF0053F30EF1DF0063F30EF1DF0072B46
:103A6000282B0725120000370137023703370837A4
:103A700009370A370B37120001011D6B1E6B1F6BD4
:103A8000206B216B226B236B246B256B266B276BC2
:103A900012001E510F0B1E6F1F510F0B1F6F205175
:103AA0000F0B206F21510F0B216F22510F0B226F33
:103AB00023510F0B236F24510F0B246F25510F0B34
:103AC000256F26510F0B266F27510F0B276F120002
:103AD0008984000EC76E220EC66E9E96C69E000E8C
:103AE000C96EFF0E9EB602D0E82EFCD79E96C69EEB
:103AF000000EC96EFF0E9EB602D0E82EFCD7C9CFCD
:103B0000A5F59E96C69E000EC96EFF0E9EB602D00B
:103B1000E82EFCD7C9CFA6F59E96C69E000EC96EAC
:103B2000FF0E9EB602D0E82EFCD7C9CFA7F59E9611
:103B3000C69E000EC96EFF0E9EB602D0E82EFCD7C0
:103B4000C9CFA8F59E96C69E000EC96EFF0E9EB602
:103B500002D0E82EFCD7C9CFA9F59E96C69E000ECE
:103B6000C96EFF0E9EB602D0E82EFCD7C9CFAAF5CB
:103B70009E96C69E000EC96EFF0E9EB602D0E82E1F
:103B8000FCD7C9CFABF589941BEC20F012008984D7
:103B9000000EC76E220EC66E9E96C69E800EC96E21
:103BA000FF0E9EB602D0E82EFCD79E96C69EA5C5F7
:103BB000C9FFFF0E9EB602D0E82EFCD79E96C69E89
:103BC000A6C5C9FFFF0E9EB602D0E82EFCD79E9672
:103BD000C69EA7C5C9FFFF0E9EB602D0E82EFCD731
:103BE0009E96C69EA8C5C9FFFF0E9EB602D0E82EBF
:103BF000FCD79E96C69EA9C5C9FFFF0E9EB602D0F1
:103C0000E82EFCD79E96C69EAAC5C9FFFF0E9EB69B
:103C100002D0E82EFCD79E96C69EABC5C9FFFF0E0C
:103C20009EB602D0E82EFCD789941BEC20F012003F
:103C30008984000EC76E220EC66E9E96C69E070E23
:103C4000C96EFF0E9EB602D0E82EFCD79E96C69E89
:103C5000000EC96EFF0E9EB602D0E82EFCD7C9CF6B
:103C6000A5F59E96C69E000EC96EFF0E9EB602D0AA
:103C7000E82EFCD7C9CFA6F59E96C69E000EC96E4B
:103C8000FF0E9EB602D0E82EFCD7C9CFA7F59E96B0
:103C9000C69E000EC96EFF0E9EB602D0E82EFCD75F
:103CA000C9CFA8F589941BEC20F08984000EC76E5B
:103CB000220EC66E9E96C69E0F0EC96EFF0E9EB653
:103CC00002D0E82EFCD79E96C69E000EC96EFF0E4F
:103CD0009EB602D0E82EFCD7C9CFADF589941BEC77
:103CE00020F012008984000EC76E220EC66E9E96CA
:103CF000C69E870EC96EFF0E9EB602D0E82EFCD778
:103D00009E96C69EA5C5C9FFFF0E9EB602D0E82EA0
:103D1000FCD79E96C69EA6C5C9FFFF0E9EB602D0D2
:103D2000E82EFCD79E96C69EA7C5C9FFFF0E9EB67D
:103D300002D0E82EFCD79E96C69EA8C5C9FFFF0EEE
:103D40009EB602D0E82EFCD789941BEC20F0898423
:103D50009E96C69E8F0EC96EFF0E9EB602D0E82EAE
:103D6000FCD79E96C69EADC5C9FFFF0E9EB602D07B
:103D7000E82EFCD789941BEC20F012008984000EF9
:103D8000C76E220EC66E9E96C69E870EC96EFF0E29
:103D90009EB602D0E82EFCD79E96C69E000EC96E37
:103DA000FF0E9EB602D0E82EFCD79E96C69E800ED1
:103DB000C96EFF0E9EB602D0E82EFCD79E96C69E18
:103DC000800EC96EFF0E9EB602D0E82EFCD79E96DE
:103DD000C69E800EC96EFF0E9EB602D0E82EFCD79E
:103DE00089941BEC20F089849E96C69E8F0EC96E26
:103DF000FF0E9EB602D0E82EFCD79E96C69E010E00
:103E0000C96EFF0E9EB602D0E82EFCD789941BEC3B
:103E100020F012008984000EC76E220EC66E9E9698
:103E2000C69E870EC96EFF0E9EB602D0E82EFCD746
:103E30009E96C69E000EC96EFF0E9EB602D0E82E5C
:103E4000FCD79E96C69E000EC96EFF0E9EB602D08F
:103E5000E82EFCD79E96C69E800EC96EFF0E9EB6BB
:103E600002D0E82EFCD79E96C69E800EC96EFF0E2D
:103E70009EB602D0E82EFCD789941BEC20F08984F2
:103E80009E96C69E8F0EC96EFF0E9EB602D0E82E7D
:103E9000FCD79E96C69E010EC96EFF0E9EB602D03E
:103EA000E82EFCD789941BEC20F012008984000EC8
:103EB000C76E220EC66E9E96C69E8F0EC96EFF0EF0
:103EC0009EB602D0E82EFCD71BEC20F09E96C69E34
:103ED000810EC96EFF0E9EB602D0E82EFCD78994E3
:103EE0001BEC20F08984000EC76E220EC66E9E96D3
:103EF000C69E8F0EC96EFF0E9EB602D0E82EFCD76E
:103F00001BEC20F09E96C69E010EC96EFF0E9EB65B
:103F100002D0E82EFCD789941BEC20F089849E9671
:103F2000C69E910EC96EFF0E9EB602D0E82EFCD73B
:103F30001BEC20F09E96C69EA50EC96EFF0E9EB687
:103F400002D0E82EFCD789941BEC20F01200898463
:103F5000000EC76E220EC66E9E96C69E8F0EC96E4E
:103F6000FF0E9EB602D0E82EFCD71BEC20F09E96EA
:103F7000C69E810EC96EFF0E9EB602D0E82EFCD7FB
:103F800089941BEC20F012008984000EC76E220E6B
:103F9000C66E9E96C69E8F0EC96EFF0E9EB602D04E
:103FA000E82EFCD71BEC20F09E96C69E010EC96E33
:103FB000FF0E9EB602D0E82EFCD789941BEC20F0B1
:103FC00012008984000EC76E220EC66E9E96C69E93
:103FD000910EC96EFF0E9EB602D0E82EFCD71BECE8
:103FE00020F09E96C69EA50EC96EFF0E9EB602D00C
:103FF000E82EFCD789941BEC20F012008984000E77
:10400000C76E220EC66E9E96C69E910EC96EFF0E9C
:104010009EB602D0E82EFCD71BEC20F09E96C69EE2
:10402000000EC96EFF0E9EB602D0E82EFCD7899412
:104030001BEC20F01200050EE82EFED71200200E19
:10404000C66E0501256B266B276B286B899A400E7F
:10405000C76E200EC66E9E96C69E030EC96EFF0EDC
:104060009EB602D0E82EFCD79E96C69E27C5C9FFF5
:10407000FF0E9EB602D0E82EFCD79E96C69E26C5A1
:10408000C9FFFF0E9EB602D0E82EFCD79E96C69EB4
:1040900025C5C9FFFF0E9EB602D0E82EFCD79E961E
:1040A000C69EC952FF0E9EB602D0E82EFCD7898A62
:1040B000C950FF0A02E166EF20F0100E2527E86ADA
:1040C0002623E86A272327A926EF20F0220EC66EB2
:1040D0001200899A400EC76E200EC66E9E96C69E2E
:1040E000060EC96EFF0E9EB602D0E82EFCD7898A56
:1040F000899A9E96C69EC70EC96EFF0E9EB602D0C6
:10410000E82EFCD7898A899A9E96C69E050EC96EAE
:10411000FF0E9EB602D0E82EFCD79E96C69EC952D0
:10412000FF0E9EB602D0E82EFCD7C9B08DEF20F06E
:10413000898A0501256B266B276B286B1200050108
:10414000FE0E2D6F0501000E2D6F68EC1DF0A5C54C
:104150002EF5A6C52FF5A7C530F5A8C531F5A9C51B
:1041600032F5AAC533F5ABC534F50784A9C159F1B9
:10417000AAC15AF1ABC15BF1ACC15CF13EC142F1E5
:104180003FC143F140C144F141C145F14AC14CF145
:104190004BC14DF10794C5EC12F000C135F501C1DA
:1041A00036F502C137F503C138F505015767E0EF71
:1041B00020F05867E0EF20F05967E0EF20F05A67F1
:1041C000E4EF20F0F2EF20F057C504F158C505F1F7
:1041D00059C506F15AC507F1010104EC1CF003BFF3
:1041E00060EF21F04CC139F54DC13AF5AFC53BF553
:1041F000B0C53CF50501100E2C6F899A400EC76EB4
:10420000200EC66E9E96C69E060EC96EFF0E9EB608
:1042100002D0E82EFCD7898A899A9E96C69E020E05
:10422000C96EFF0E9EB602D0E82EFCD79E96C69EA3
:1042300027C5C9FFFF0E9EB602D0E82EFCD79E967A
:10424000C69E26C5C9FFFF0E9EB602D0E82EFCD73B
:104250009E96C69E25C5C9FFFF0E9EB602D0E82ECB
:10426000FCD725EE2DF02C2F02D042EF21F09E96A8
:10427000C69EDECFC9FFFF0E9EB602D0E82EFCD749
:1042800033EF21F0898A899A9E96C69E050EC96EE3
:10429000FF0E9EB602D0E82EFCD79E96C69EC9524F
:1042A000FF0E9EB602D0E82EFCD7C9B04DEF21F02C
:1042B000898A0501100E2527E86A2623E86A272344
:1042C000120019C502F51AC503F525EE5FF00501C8
:1042D0002C6B16EE00F005010251E1260351D8B017
:1042E0000329E226E7CFE8FF2C0A06E12CC5DEFF12
:1042F00005012C6B84EF21F0E7CFE8FF2A0A0CE0E0
:10430000E7CFDEFF05012C2B0501032B023F03073E
:10431000030E031769EF21F005012D6B2E6B2F6B38
:10432000306B316B326B336B346B356B366B376B99
:10433000386B396B3A6B3B6B3C6B3D6B3E6B3F6B49
:10434000406B416B426B436B446B456B466B476BF9
:10435000486B496B4A6B4B6B4C6BDDCFE8FF05013B
:104360002C5105E0DDCFE8FF2C2FB2EF21F0050145
:10437000DDCF2CF52C5105E0DDCFE8FF2C2FBCEF75
:1043800021F00501DDCF2CF52C5105E0DDCFE8FF54
:104390002C2FC6EF21F011EE27F001013CEC1DF0AF
:1043A0000501DDCF2CF52C5105E0DDCFE5FF2C2FED
:1043B000D5EF21F0010149EC1DF0C0EC1CF000C16B
:1043C0002EF501C12FF502C130F50501DDCF2CF529
:1043D0002C5105E0DDCFE8FF2C2FEAEF21F005019D
:1043E000DDCF2CF52C5105E0DDCFE8FF2C2FF4EFCD
:1043F00021F00501DDCF2CF52C5107E0DDCFE8FFE2
:10440000E8A82D852C2FFEEF21F011EE27F00101F9
:104410003CEC1DF00501DDCF2CF52C5114E0DDCF77
:10442000E5FFDDCFE5FFDDCFE5FFDDCFE5FFDDCF4C
:10443000E8FFDDCFE5FFDDCFE5FFDDCFE5FFDDCF39
:10444000E5FFDDCFE5FF010149EC1DF0C0EC1CF0FC
:1044500000C138F501C139F502C13AF503C13BF598
:104460000501DDCF2CF52C5107E0DDCFE8FFE8A8F2
:104470002D832C2F35EF22F011EE27F001013CECBB
:104480001DF00501DDCF2CF52C5105E0DDCFE5FF5A
:104490002C2F46EF22F0010122C123F121C122F18C
:1044A00020C121F11FC120F149EC1DF0C0EC1CF02E
:1044B00000C134F501C135F502C136F503C137F548
:1044C0000501DDCF2CF52C5107E0DDCFE8FF2C2FC7
:1044D00065EF22F0E8B02D8711EE27F001013CECEA
:1044E0001DF0DDCFE8FFDDCFE8FFDDCFE8FFDDCF5A
:1044F000E8FFDDCFE8FFDDCFE5FFDDCFE5FFDDCF76
:10450000E5FFDDCFE5FFDDCFE5FFDDCFE5FF49ECE2
:104510001DF0C0EC1CF000C131F501C132F502C143
:1045200033F5078455C159F156C15AF157C15BF1B2
:1045300058C15CF13EC142F13FC143F140C144F179
:1045400041C145F14AC14CF14BC14DF10794C5EC55
:1045500012F000C13CF501C13DF502C13EF503C1B9
:104560003FF5120021C500F122C501F123C502F17A
:1045700024C503F1899A400EC76E200EC66E9E9622
:10458000C69E0B0EC96EFF0E9EB602D0E82EFCD75B
:104590009E96C69E02C1C9FFFF0E9EB602D0E82EAF
:1045A000FCD79E96C69E01C1C9FFFF0E9EB602D0E3
:1045B000E82EFCD79E96C69E00C1C9FFFF0E9EB690
:1045C00002D0E82EFCD79E96C69EC952FF0E9EB61C
:1045D00002D0E82EFCD725EE2DF00501100E2C6F31
:1045E0009E96C69EC952FF0E9EB602D0E82EFCD7FC
:1045F000C9CFDEFF2C2FF0EF22F0898A1200899AB2
:10460000400EC76E200EC66E9E96C69E900EC96E58
:10461000FF0E9EB602D0E82EFCD79E96C69E000ED8
:10462000C96EFF0E9EB602D0E82EFCD79E96C69E9F
:10463000000EC96EFF0E9EB602D0E82EFCD79E96E5
:10464000C69E000EC96EFF0E9EB602D0E82EFCD7A5
:104650009E96C69EC952FF0E9EB602D0E82EFCD78B
:10466000C9CF2DF59E96C69EC952FF0E9EB602D0AA
:10467000E82EFCD7C9CF2EF5898A120018EC1EF05F
:10468000F29CF29E8B948A86899CC69AC2908A94E8
:10469000898A9482948C720ED36ED3A4FED78996A5
:1046A0008A909390FF0EE8CF00F0E82EFED7002E00
:1046B000FCD78150F294F29A9E909D909E929D928A
:0E46C000F298F292F290F286F28E0300FF0062
:10BF0000E844F926000C160C2B0C3F0C520C640C68
:10BF1000760C860C960CA50CB30CC10CCF0CDC0C6B
:06BF2000E80CF40C000C1B
:00000001FF
